:10000000000C2500D10C02006607040A6606060AE9
:1000100061006607090A01022E00220C8E00030609
:10002000040A1A0C8E000306180A080CE501040ADB
:10003000D70C020058029B01890143066D0AC304D4
:100040007C00700067007E007F007A00BA027B00AF
:10005000770068043F0C0600300C24006A00A305FA
:100060000509A30443062F0A0F0220003F0C840158
:100070003F0E43066D0AA402AA022F0A0702E201FC
:10008000000800080008000802080308050807081F
:100090000A080D08120816081C082208290830084A
:1000A000380841084A0854085F086A087608830837
:1000B00090089E08AD08BC08CC08DC08ED08FF08D5
:1000C000090C2E00400003042F000F032D0303062C
:1000D000CC01EE02640A2C0000080400FF0C2D0085
:1000E0002E002F00090C24000B0C3D007F0048045B
:1000F000000099094806810AB7096606C805800A02
:10010000810AFC0C3F024306910ADF01FD028D0AC1
:100110000306C80ABD020000760ADF0203065B0B75
:10012000760A0000930AC806BF02C804FE03770AD5
:100130002A0A66070008BF027E004805B70966075D
:100140000008BF02000009029B0138007802A806DF
:10015000B20A3E0930000304E80630034804DF0316
:10016000990A2A0A0000B40AB50AB60AAE0AB80A01
:10017000B90ABA0ABB0ABC0ABD0ABE0A00000008D6
:10018000100C8400070E43065A0BC806BF02CC0AA7
:10019000090C3D00A4027F004804C80499094806E0
:1001A000D80AB7096606C805000000000000000074
:1001B000FC0C3F024306C00ADF01FD02270B0306C9
:1001C000C80A79000A028B018C018D018E018F0112
:1001D0004307440B6A026B026C026D026E02B709A0
:1001E000E400080C0600A4050A02EA07150B9101B9
:1001F00043070E0B0B02920143070E0B2C0C24003D
:10020000B4070E0B28060E0B0000A3054F0A080BBF
:10021000090B0C0B28066D0A0000210B0A02F00ED8
:10022000700F43076D0AA305E90A4306070BB407DD
:10023000900143060A0B13027F0E2804430728058A
:100240008A0143070E0B2B0C2400A3054F0A000064
:100250006003DF02CB0A5D0B970C2C00040C8700B7
:100260002D0060092C032D032C032D032C032D03DB
:100270002C032D030C063F0B010CCD010306FF0CD4
:10028000A40430006D0A000000000000000000001F
:10029000B70900000000000000000000000000009E
:1002A000000000006D0A00000000000000000000D7
:1002B000000000000000B902F9075F0B000A430BC1
:10040000840C3500310A800C060A830C3500A00CE0
:10041000C6042900080C2800E6046903C604030684
:10042000C6050000E605E8020C0A0000E60400002C
:10043000C60500000000E605C606F504E604F5075B
:10044000470A15020F0EE2012B0A2E0A470A2B0A51
:10045000310A360A470AB5020A02090AB5020F0232
:10046000090AE605C605B502A10C080AC605000082
:10047000E605080C2800E6050305C60703046F031C
:10048000E604C605E8023B0AE6050000E604C604E9
:10049000E6054A0A4B0AC605F5070008010880036D
:1004A0002F000F03070EE201870ACB0B8A0B980B74
:1004B0005F0B570BEA0B0B02F90F4306170B0002F9
:1004C0002A00A40200022B00A40200022C00EE0A63
:1004D0002400070C4C017E098C07750A6C0620016C
:1004E000FF0F6C0760010402FB0A400143067B0A10
:1004F0006C06280BEA0B6C07280BEA0BE2010108DB
:10050000020804080808100820084008800880062F
:10051000BE0BEA0B8007A80A08069B0A54069D0A30
:10052000E807940A680600085702690116022901C3
:10053000E805680500085406900AE806A10A68065E
:1005400000085602690117022901E804680500083D
:10055000680700085602690157026901680400082B
:1005600048046804000F43063008100F43063108A2
:10057000010F43063208030F430633080E0F4306EC
:1005800034083C0F43063608010F43063708030FB3
:1005900043063808010F43063908070F43063A0897
:1005A000010F43063B08030F43063C08010F4306B7
:1005B0003D080F0F43063E08010F43063F0868053C
:1005C0002F0F43060208010F43060D086804480573
:1005D000FF0804020F0E0C0F43073F0B0B02B0097C
:1005E0004806EA0B68066A07F70A3500350C4A0721
:1005F000680A6A071C0B0F0E2A0005096800000232
:100600008F014306A30443062C0A00022F00D406E0
:100610000F0BD405ED0BF4060F0BF405ED0B0309DE
:1006200043060F0B6800A304D404F404000A0A0272
:100630002000400075001F0B68063D0B0F0E2A00BE
:100640000509680000028F014307A30443076D0AF0
:10065000C3062C0BC305ED0BFF07EA0B310C26007C
:10066000090C2E006F000400EF03340BEE02320B76
:100670006600C304A404A3046D0A8001240B0A02CB
:100680007D0FF70E4306500B010F4306540B0A0271
:10069000070ED501B0094806EA0B6A071C0BFB0AD6
:1006A000EB0003046B036B030A02070E4D0B80077C
:1006B000EA0B8003F00EA4043B010F0F670B8A09BD
:1006C0008006340500020F0EA4043B01F00F5B010D
:1006D0003B002E0097012F00A405750015027E092E
:1006E0004F0143077C0BB50275076E0B090226000C
:1006F000A4041B023700EA0B380CD50124001502B4
:100700007E094E014306870B00022901730B40024C
:100710006901730B14069A0BF3069C0B0807A60BD2
:10072000A4041C0243060804A40470006700EA0B3A
:1007300014068C0BF3068E0B0806A60BA4041C02F1
:1007400043060805A40470006700EA0BA8044003F0
:100750001E0E2700800607053407070434078A09A0
:1007600007024306BD0BFD0E4306BD0B9406EA0BC4
:10077000A3042C0B080C06006600EA0B0C023300E5
:100780000002120F4306F304010F4306F305330C76
:1007900024001302FB0A00023F0F4307EA0BA402E6
:1007A000E006D90B1406DB0BF306DD0B0806900BF5
:1007B000DF0B1406D40BF306D60B08079E0B0003C1
:1007C0002F000F031F0E27003405A8054003A404C3
:1007D0003000EA0BD404F404C304A304A4046D0A97
:0207FE00700C7D
:021FFE00EE0FE4
:00000001FF
